:060000000C946E010C944B
:10000600F2020C9495020C9400000C9400000C94DF
:1000160000000C9400000C94FD030C9400000C945A
:1000260000000C9400000C942B030C9400000C941C
:1000360000000C9400000C9443030C9400000C94F4
:1000460000000C9400000C9400000C940000040EB8
:100056001F15040404041B11000A1B1B1B1B0404AC
:100066000404151F0E041B1B1B1B0A00111B1F1B60
:100076000A110A1B1F7FD804F60414053205500521
:100086006E058C05AA05C805E60504062206400687
:100096005E067C069A06B806D606F40612073007F0
:1000A6004E076C076C076C076C076C076C076C07D0
:1000B6006C076C076C07640001000000000000007C
:1000C600000000000000000000000000000000002A
:1000D600000000001027E80364000A000100001079
:1000E6000001100001004B616C69627269657275EE
:1000F6006E670020202D2020202020454E540053DE
:1001060074726F6D73656E736F72204E756C6C6171
:1001160062676C656963680020414443206C6F77B1
:100126002020200020414443206869676820202061
:10013600002057657274652067657370656963682A
:1001460065727420005374726F6D204C6F77204B6C
:10015600616C6962722E00204B6F72722E20202015
:10016600002D002C00300020412020200053747206
:100176006F6D2048696768204B616C6962722E005A
:100186005370616E6E756E6773204B616C69627237
:100196002E0020562020200054656D706572617413
:1001A6007572732E2030274300204144432054317A
:1001B6003A20002020202000204144432054323A97
:1001C600200054656D7031204B616C6962722E207F
:1001D6003130302743002027432020200054656D0E
:1001E6007032204B616C6962722E203130302743A9
:1001F6000050633A20200045696E00417573004E39
:10020600756C6C413A2B004C6F673A20004675744A
:1002160075726520202000426C6174743A20313A70
:10022600004B616E3A200053746172744D3A003E81
:10023600003B00206E6F2043656C6C004D0056003D
:10024600410020550054313D00DF430054323D004B
:100256002054693A0056312000566D20005632204F
:1002660000202D00207C00202F00506172616D65FA
:1002760074657200202020202020454E5400496ECF
:10028600697469616C69736174696F6E20696E2047
:1002960050726F6772657373004C69506F20566FAA
:1002A6006C746D657465720054656C656D65747209
:1002B6006965005665722E20322E320032332E309A
:1002C600332E32303130000002000204BC0001003F
:1002D6000504BE000000F894EE27ECBBF1E0FBBF7E
:1002E600EBBFE5BFF8E1F1BDE1BD8DE0A2E0BB27C4
:1002F600ED938A95E9F780E098E0A0E6ED93019703
:10030600E9F7EEECF2E085919591009761F0A59101
:10031600B59105901590BF01F00105900D920197DA
:10032600E1F7FB01F0CFEFE5EDBFE8E0EEBFC0E699
:10033600D2E00C945D151A930A93EA81EE0FEE0F44
:10034600EE0FE0640E2F10E0183070F40A93039558
:10035600EC81FD813196EC83FD833197E491EA933C
:100366000E9438181F5FF0CF1981088125960895DD
:10037600000000000000C19A00000000000000001C
:1003860000000000C1980000000000000895AF932F
:10039600AFB7AF93BF93A8E0B881AA23C9F0AA95D7
:1003A6008894BB1F18F0C09804D0F7CFC09A01D02C
:1003B600F4CF000000000000C19A00000000000019
:1003C600000000000000C198000000000000089531
:1003D600C098BF91AF91AFBFAF9121960895C298D3
:1003E6000E9423190E942719C29A0000C2980E94EF
:1003F6002319EBE8EA930E94CA01C29A0000E0E0E2
:10040600E093DD030895249784E0A0E0B0E0E0ECFB
:10041600F0E00E94A421E0E0E8830E942B190E94EC
:10042600301948F40E943719A981EA27E983E8813F
:10043600EF5FE883F2CFE981EA83E981E07FE98330
:10044600E295EF70E983A981AA3010F0E95C02C059
:10045600E981E063E983FE013296DF01EC91EF70FA
:10046600EC93AA81AA3020F0EA81E95CEA8306C00F
:10047600FE013296DF01EC91E063EC93E0E0EB8362
:100486000E942B190E943D194BC0249784E0A0E0DE
:10049600B0E0E4ECF0E00E94A421E0E6F2E00E9485
:1004A6004319E883E4500E944719EA83E881E35040
:1004B6000E944719EB83AA81AA3318F0EA81E75311
:1004C60002C0EA81E053EA83AB81AA3318F0EB81DC
:1004D600E75302C0EB81E053EB83EA81EF70EA83D6
:1004E600FE013396DF01EC91EF70EC93EA81E29521
:1004F600E07FEA83EB81AA81EA2BEA83E0E0E983E5
:10050600E881E450A981AE1750F4E9810E944719A9
:10051600AA81EA27EA83E981EF5FE983F1CFEA81DD
:10052600249608950E944C190E94982100E010E03C
:1005360030E0E0E0E093DE03C098C298E0E0EA93A2
:100546000E94CA01E0E0EA930E94CA0110E0183056
:1005560060F4B39B05C0E02FEE0FE1600E2F01C0E3
:10056600000F0E94BB011F5FF2CFC29A0000043247
:1005760021F0A091DD03AE3750F0E1E0E093DD031A
:10058600E4E2E0936002E0E0E09361020CC00E94C6
:100596005A190083E091DD03EF5FE093DD030E94CB
:1005A6005A19A0E0A0830A30A1F40E94F2010E9429
:1005B60048023E2F303051F4EFEDF2E0FA93EA9321
:1005C600E0E6F2E00E946019689420F8E0E0E0932B
:1005D600DD030E949F2124960E9464191895AF930B
:1005E600A2B7BF93BFB7BF93B091EA03A093EA0344
:1005F600AB1BA093EE03A091E703B091EB03A0938E
:10060600EB03AB0BA093EF03A091E803B091EC03CF
:10061600A093EC03AB0BA093F003A091E903B09178
:10062600ED03A093ED03AB0BA093F103A091FE03A2
:10063600A395A093FE0329F4B091FF03B395B0935D
:10064600FF03BF91BFBFBF91AF91689424F818957F
:10065600AF93AFB7AF93A091E703A395A093E7033A
:1006660059F4A091E803A395A093E80329F4A09177
:10067600E903A395A093E903AF91AFBFAF91189596
:100686000A92AA93BA93EA93FA93EFB7EA93082CDD
:10069600092891F0F40131974F01A8EAB4E0A60DBC
:1006A600B71DEC91ECB9F30131963F01E030A1E0C2
:1006B600FA0711F466247724E991EFBFF991E991DD
:1006C600B991A99109901895E0E0F1E0E815F905CE
:1006D600D9F3F894082C092811F45D9912C0F20197
:1006E600E855FB4FA881A083F20131962F01E03037
:1006F600A1E0FA0711F444245524F40131964F0180
:1007060002C0E881ECB978942196089522970E9458
:1007160072190E944721EF2FF0E0E983FE0131961E
:10072600DF01EC91E06AEC930E9472190490088252
:10073600C2980E942719ECE6EA930E94CA01C29A5F
:100746000000C298E2ECEA930E94CA010E947C195A
:10075600C29A0000C298E981EA930E94CA01E88120
:10076600EA930E94CA01C29A0000C2980E947C19AC
:10077600E0E8EA930E94CA01C29A0000C2980E9469
:100786007C19E1E8EA930E94CA01C29A0000C29865
:100796000E9423190E942719C29A0000C2980E943B
:1007A6002319EBE8EA930E94CA01C29A0000C29894
:1007B600E4ECEA930E94CA01ECEAEA930E94CA01B9
:1007C600C29A0000C298E8ECEA930E94CA01E1E9E5
:1007D600EA930E94CA01C29A0000C298E6ECEA9324
:1007E6000E94CA01EFEBEA930E94CA01C29A000076
:1007F600229608950E944C19E091E403F091E503D6
:100806003196E093E403F093E503E0E024FCE1E0B5
:10081600E130A8F0E091EE03F091EF036091F00370
:100826007091F1030E9480190E946A200E94891922
:10083600E091F903EF5FE093F903E89424F8A091BF
:10084600E403B091E503989748F1E091FE03F09137
:10085600FF03E0930004F0930104E0E0E093FE035D
:10086600E093FF03E0E0E093E403E093E50368949C
:1008760021F8E091F803EF5FE093F803E091DE03DF
:10088600EF5FE093DE03A091DE03A43038F00E9410
:1008960089030E94F201E0E0E093DE030E946419FE
:1008A6001895E881E06CE7B985E38A95F1F7369A01
:1008B600349BFECF349AE4B1F5B121960895000039
:1008C6000000C7980000000000000000C79A000062
:1008D600000008952297E0B3E07FE883EAE0F0E0C5
:1008E6000E949219E0B3E07FE983A881EA1711F428
:1008F600E88117C0E0E015C01A9310E010E0183048
:1009060070F4E981E078E03811F4DF9A01C0DF98ED
:100916000E946204E981EE0FE9831F5FF0CFDF9A40
:100926001881229608950E94982120E030E0EC81FB
:10093600E770EC83DF9A0E949619EC81E069EA93EE
:100946000E947F04C59A00000E949F19E0E20E945F
:10095600A4190E94AB190E94B019A9F00E94B619F9
:10096600E091E203E03D39F40E94BB1918F0E0E0A3
:10097600E093A70408C0E03B31F40E94C41919F4BF
:10098600E4E0E093A704E8E2F0E00E949219B69B47
:1009960002C00E94CB19B69B05C020E030E00E9441
:1009A600CE190FC0E8E5EA930E947F0410E01031EB
:1009B60040F4B6992160220F331F0E9462041F5F24
:1009C600F6CFC59A0000F9010E949F212596089549
:1009D6001A93C5980000DF9A10E0123220F40E94A4
:1009E60062041F5FFACFC59A0000199108952197F6
:1009F600E0E0E883A881A43080F50E949619E8819A
:100A0600E069EA930E947F04C59A00000E949F193C
:100A1600E0E80E94A4190E94CB19B69B06C0E4E642
:100A2600F0E00E9492190E94CE19C59A00000E9419
:100A36009F19E0EA0E94A4190E94CB19B69B06C032
:100A4600E4E6F0E00E9492190E94CE19C59A0000D1
:100A5600E881EF5FE8830C94FD04219608951A93CC
:100A660010E01630D8F4E12F0E94D519EA0FFB1FCB
:100A76000F010E94DB190E94E219ED93FC930E947C
:100A8600DB19EA0FFB1FFF93EF931A930E9496045C
:100A9600AF91BF91ED93FC931F5FE3CF199108953A
:100AA6006E9784E0AAE1B0E0E8ECF0E00E94A421B1
:100AB6000E94962110E020E030E040E050E00E94E5
:100AC600B6190E94E819ECEEF0E00E94EF190E94B8
:100AD600F319E9EFF0E00E94EF190E94B01931F026
:100AE600A091E203A03011F0A03F19F40E94AB19C7
:100AF600F4CFA091E203A03711F00C94D6080E941F
:100B0600E819E5E0F1E00E94EF190E94F9190E9448
:100B1600FC19A091E203A03751F10E94001A10E0DF
:100B26001A3030F40E940B1A0E940F1A1F5FF8CF7A
:100B36000E942C1A0E94311A0E94361A0E943F1AED
:100B46000E94441A0E944A1A0E944F1AEEE1F1E0EE
:100B56000E945C1A0E94661A0E946C1A0E944F1A22
:100B6600EAE2F1E00E945C1A0E94AB19D2CF0E9421
:100B7600711A19F40E94791A21F00E94841A0E94AF
:100B86008A1A0E94E8190E94901A0E94F9190E9476
:100B9600E819EBE4F1E00E94EF190E94F9190E94AE
:100BA600AB190E94B619A091E203A03711F40C9478
:100BB6003C060E94AB190E94B019A1F0A091E20375
:100BC600A03D29F40E94931A31960E94981AA0918A
:100BD600E203A03B29F40E94931A31970E94981AC7
:100BE6000E94B6190E940B1A0E949D1A0E944A1A68
:100BF6000E94A41A0E94AB1A0E94931A0E94A41A79
:100C06000E94B21A0E94B91A0E94BE1A0E94C51A00
:100C16000E94931A0E944F1A0E94CA1A0E94661ACC
:100C26000E94CD1A2CF40E94D11A0E94D41A02C036
:100C36000E94DA1A0E94DD1A0E94E31A14F40E9436
:100C4600F01A0E94F61A0E9460190E94051B0E9463
:100C56000A1B0E94111B24F40E94051B0E94181BEC
:100C66000E94F61A0E941E1BEDE6F1E00E945C1A35
:100C76009ACFA4E0B0E00E945D21A0912B04B09130
:100C86002C04EA17FB0731F00E94931AA4E0B0E0A7
:100C96000E946D210E94E8190E94901A0E94F9197B
:100CA6000E94E819E3E7F1E00E94EF190E94F919A2
:100CB6000E94AB190E94B619A091E203A03711F465
:100CC6000C94C4060E94AB190E94B019A1F0A09121
:100CD600E203A03D29F40E94231B31960E94281BA3
:100CE600A091E203A03B29F40E94231B31970E94A6
:100CF600281B0E94B619E1E00E942D1B0E946C1A67
:100D06000E94A41A0E94AB1A0E94231B0E94A41AD6
:100D16000E94B21A0E94B91A0E94311B0E94C51A7B
:100D26000E94231B0E944F1A0E94CA1A0E94661A2A
:100D36000E94CD1A2CF40E94D11A0E94D41A02C025
:100D46000E94DA1A0E94DD1A0E94E31A14F40E9425
:100D5600F01A0E94F61A0E9460190E94051B0E9452
:100D66000A1B0E94111B24F40E94051B0E94181BDB
:100D76000E94F61A0E941E1BEDE6F1E00E945C1A24
:100D86009BCFA0E0B0E00E945D21A0912704B09126
:100D96002804EA17FB0731F00E94231BA0E0B0E00D
:100DA6000E946D210E94E8190E94901A0E94F9196A
:100DB6000E94E819E6E8F1E00E94EF190E94F9198D
:100DC6000E94AB190E94B619A091E203A03711F454
:100DD6000C9442070E94AB190E94B019A1F0A09191
:100DE600E203A03D29F40E94381B31960E943D1B68
:100DF600A091E203A03B29F40E94381B31970E9480
:100E06003D1B0E94B619E4E00E942D1B0E94381B70
:100E16000E94B91A662777270E94B21A0E94B91A49
:100E26000E94421B0E94C51A0E94381B0E944F1A3C
:100E36000E94CA1A0E94491B0E94F720AF010E9415
:100E46004F1B4A30E0E05E0724F40E94DA1A0E9443
:100E5600F01A0E94F61A0E9460190E94051B0E9451
:100E6600551B0E94491B0E940321AF010E94F61ADE
:100E76000E941E1BE8E9F1E00E945C1AA5CFA0E1E2
:100E8600B0E00E945D21A0913704B0913804EA17C2
:100E9600FB0731F00E94381BA0E1B0E00E946D21F3
:100EA6000E94E8190E94901A0E94F9190E94E819F6
:100EB600EEE9F1E00E94EF190E94F9190E94FC196F
:100EC600A091E203A03711F40C94BC07E0E0F0E037
:100ED6000E945B1BE1E3F4E0A0E0B0E0A083B183F5
:100EE60010E01A30D8F4E2E0EA930E9454049F011D
:100EF600E3E0EA930E945404AF01F901A0912F04A4
:100F0600B0913004EA0FFB1F0E945B1B0E94601B1E
:100F1600E40FF51F0E94651B1F5FE3CFA0912F040E
:100F2600B09130040E94311A0E945B1BA0913104DB
:100F3600B09132040E94311A0E94651B0E946A1BFE
:100F4600EFEAF1E00E94EF190E946F1B0E944F1A10
:100F56000E94741B0E94791BEEEBF1E00E94EF19D0
:100F66000E94601B0E944F1A0E94741B0E94AB19BC
:100F7600A7CFA8E0B0E00E945D21DF010E946F1BB1
:100F8600EA17FB0751F4AAE0B0E00E945D21DF01F9
:100F96000E94601BEA17FB0761F00E946F1BA8E026
:100FA600B0E00E946D21AAE0B0E00E94601B0E94A2
:100FB6006D210E94E8190E94901A0E94F9190E9458
:100FC600E819E8ECF1E00E94EF190E94F9190E9475
:100FD600AB190E94B619A091E203A03711F40C9444
:100FE60047080E94AB190E94B019D1F0A091E20304
:100FF600A03D41F4A3E3B4E0ED91FD913197FE935A
:10100600EE933196A091E203A03B41F4A3E3B4E052
:10101600ED91FD913196FE93EE9331970E94B619AC
:10102600E2E00E942D1B0E946F1B0E94A41A0E94E0
:10103600AB1A0E947F1B0E94851B0E94A41A0E9465
:10104600F7200E94C51A0E94851B0E944F1A0E9413
:10105600CA1A0E94661A0E94CD1A2CF40E94D11A4E
:101066000E94D41A02C00E94DA1A0E944F1B0E94E4
:101076008A1BFE0138960E9460190E94051BECED42
:10108600F1E00E945C1AA7CFACE0B0E00E945D21BF
:10109600DF010E94851BEA17FB0731F00E94851BC2
:1010A600ACE0B0E00E946D210E94E8190E94901AFF
:1010B6000E94F9190E94E819E3EEF1E00E94EF1987
:1010C6000E94F9190E94AB190E94B619A091E20379
:1010D600A03711F40C94C0080E94AB190E94B019F5
:1010E600C1F0A091E203A03D39F4A5E3B4E0ED918F
:1010F600FD913197FE93EE93A091E203A03B39F464
:10110600A5E3B4E0ED91FD913196FE93EE930E9436
:10111600B619E3E00E942D1B0E94601B0E94A41AD0
:101126000E94AB1A0E947F1B0E94951B0E94A41A64
:101136000E94F7200E94C51A0E94951B0E944F1A12
:101146000E94CA1A0E94661A0E94CD1A2CF40E94A6
:10115600D11A0E94D41A02C00E94DA1A0E944F1BAA
:101166000E948A1BFE0138960E9460190E94051B88
:10117600ECEDF1E00E945C1AA9CFAEE0B0E00E946F
:101186005D21DF010E94951BEA17FB0731F0AEE0F7
:10119600B0E00E94951B0E946D210E94E8190E94F2
:1011A600901A0E94F9190E949D21A49608952497E9
:1011B6000E948518E1E00E949A1BE7EFF1E00E9489
:1011C600EF19E0E023FCE1E0E13018F0EDEFF1E0AB
:1011D60002C0E1E0F2E0FA93EA930E94BD18EBE068
:1011E6000E949A1BE5E0F2E00E94EF190E946A1B3A
:1011F600EDE0F2E00E94EF19E0E022FCE1E0E130F0
:1012060018F0EDEFF1E002C0E1E0F2E0FA93EA93C4
:101216000E94BD18EBE00E949F1BE3E1F2E00E94F2
:10122600EF190E94791BEDE1F2E00E94EF19A091FF
:101236000504AA3010F40E94DA1AE09105040E940F
:10124600A41BE9E6F1E00E94EF19A0910404AA307C
:1012560020F4EBE6F1E00E94EF19E09104040E940D
:10126600A41BE1E00E94B21BE7E2F2E00E94EF1944
:10127600E091DF030E94A41BEBE00E94B21BEDE2AB
:10128600F2E00E94EF19E091E1030E94A41BEC81B9
:10129600E03019F4E0E0EA932DC0E13021F4EAE011
:1012A600EA93E0E027C0E23021F4E0E0EA93E1E0EF
:1012B60021C0E33021F4EAE0EA93E1E01BC0E43028
:1012C60021F4E9E0EA93E2E015C0E53021F4ECE030
:1012D600EA93E2E00FC0E63021F4EDE0EA93E2E0C3
:1012E60009C0E73011F4E0E003C0E83031F4EAE089
:1012F600EA93E3E0EA930E945D18E5E3F2E00E94D8
:10130600EF19259608950E94962100E010E0A0911D
:10131600E203A03E11F40C94E20A0E94AB190E946B
:10132600B01911F40C94E10A0E94B619A091E203D7
:10133600A03D11F00C941A0AE12FE03021F46894D4
:101346000E94B71B74C0E130F1F40E94001A00E05D
:101356000A3030F40E940B1A0E940F1A0F5FF8CF62
:101366000E942C1A0E94311A0E94361A0E943F1AB5
:101376000E94711A11F00E94841A0E94791A11F0C3
:101386000E948A1A54C0E23021F4689422F8DE9A48
:101396004EC0E33009F44BC0E43081F4E09105041B
:1013A600EF5FE0930504A0910504A53130F0E0E07D
:1013B600E0930504E1E0E093040439C0E53069F404
:1013C600E0910404E65FE0930404A0910404A436CB
:1013D60018F0E0E0E09304042AC0E63059F4E09106
:1013E6000404EF5F0E94BE1BA43618F0E0E0E09311
:1013F60004041DC0E73069F4E091DF03EF5FE0937A
:10140600DF03A091DF03A73118F0E0E0E093DF03EC
:101416000EC0E83061F4E091E103EF5FE093E10391
:10142600A091E103A53018F0E0E0E093E103A0917C
:10143600E203A03B11F00C947A0AE12FE03021F48C
:10144600E8940E94B71B53C0E23021F4E89422F8D6
:10145600DE984DC0E430A9F4E0910504E150E09334
:101466000504E03019F4E3E6E0930404E091050492
:10147600EF5F31F4E4E1E0930504E0E0E093040477
:1014860036C0E53059F4E0910404EA500E94BE1BD0
:10149600A03818F0E3E6E093040429C0E63059F4D6
:1014A600E0910404E1500E94BE1BA03818F0E3E668
:1014B600E09304041CC0E73059F4E091DF03E150E7
:1014C600E093DF03EF5F19F4E6E1E093DF030FC07B
:1014D600E83069F4E091E103E150E093E103EF5F66
:1014E600E091E103EF5F19F4E4E0E093E103A091FA
:1014F600E203A03711F00C94DE0AE12FE03011F47C
:101506001F5F59C0E13011F41F5F55C0E23011F47E
:101516001F5F51C0E33011F41F5F4DC0E43011F07E
:10152600E53009F402C0E63019F51F5FE0910504C5
:10153600F0E00E94C31B0E94C81BE4E60E94AF2095
:10154600DF01E0910404F0E0EA0FFB1F0E94C31BD9
:10155600A3E1B0E00E945D210E94C81BEA17FB07C9
:1015660031F00E94CD1BA3E1B0E00E946D2123C0A3
:10157600E73081F41F5FA5E1B0E00E946121A091F0
:10158600DF03EA1731F0E091DF03A5E1B0E00E9446
:10159600752111C0E83079F410E0A2E1B0E00E94B4
:1015A6006121A091E103EA1731F0E091E103A2E1A4
:1015B600B0E00E9475211A930E94DA08A8CE0E9414
:1015C6009D2126960895219781E0A0E0B0E0ECECFD
:1015D600F0E00E94A421E0E0E0939A04E0939B04EB
:1015E600E0939C04E0939D04E0E0E0931E04E8830E
:1015F600A881A630F0F40E94D21B0E94DB1B66274E
:1016060077270E94E31BEA0FFB1F0E94DB1B0E9449
:10161600EC1B0E94F11BEA0FFB1F0F01E8810E94E1
:10162600D5190E94E2190E94EC1BE881EF5FE8835E
:10163600DFCFE6E0E883A881A13010F40C948F0B8D
:101646000E94F81B7F936F93FF93EF930E94041CF5
:101656000E943C21AF91BF918F919F910E948C2156
:101666003CF40E94041CE0E0F0E060E070E018C08A
:101676000E940D1CFF93EF930E94041C0E943C21C4
:101686007F936F93FF93EF930E94F81BAF91BF91E7
:101696008F919F910E9450210E946F20AF91BF9120
:1016A6000E9442210E94161C7F936F93FF93EF9333
:1016B6000E94F11B0E94221CAF91BF918F919F91B6
:1016C6000E948C214CF40E94F11BAE0FBF1FE0E07C
:1016D600F0E060E070E01AC00E94F11BEA0FFB1F09
:1016E600FF93EF930E94F11B0E94221C7F936F933E
:1016F600FF93EF930E94161CAF91BF918F919F911C
:101706000E9450210E946F20AF91BF910E944221FA
:10171600E881E150E8838FCFE0E0E883A881A63036
:1017260010F00C94F40BF8940E940D1CFF93EF93A9
:101736000E94041C0E943C210E94271CAF91BF916D
:101746000E9442210E94D21BFF93EF930E94361CF7
:101756000E94271CAF91BF910E9442210E94F11B5B
:10176600EA0FFB1FFF93EF930E94F11B0E94221CBE
:101776000E94271CAF91BF910E94E31B0E94221C6E
:10178600DF01CB01E0919A04F0919B0460919C04E7
:1017960070919D040E948C217CF40E94041C0E947E
:1017A6003C21E0939A04F0939B0460939C0470930D
:1017B6009D04E881E0939E040E94041C0E943C2143
:1017C600E53FA1E0FA07A0E06A07A0E07A071CF06F
:1017D600E881E0931E047894E881EF5FE8830C9437
:1017E600910BE2E0EA930E945404662777270E9451
:1017F6003D1C0E94461C0E944F1C59F4E0E0E093F9
:101806009F04E093A004E093A104E093A2040C9447
:101816001E0CF8940E946F1B0E94461C0E94571CC7
:10182600DF01CB010E94851B0E948A200E94F720BF
:101836000E943D1C7894E3E0EA930E9454046627D4
:1018460077270E94621C0E946B1C0E944F1C59F451
:10185600E0E0E093A304E093A404E093A504E093FE
:10186600A6040C94480CF8940E94601B0E946B1C02
:101876000E94571CDF01CB010E94951B0E948A2003
:101886000E94F7200E94621C7894A0910004B091F7
:101896000104139750F4E0E0E093FA03E093FB03AE
:1018A600E093FC03E093FD0334C0A0910004B091E3
:1018B6000104AE35E1E0BE07C0F4E091F9030E94F1
:1018C6008019FF27662777270E94D2200E94891950
:1018D6000E94CD1B0E948019662777270E948F20C1
:1018E600A0E0BFE288E699E510C0E0910004F0911F
:1018F6000104662777270E94741C0E947D1CE0E77E
:10190600F7E160E070E00E94861C0E94D2200E94EF
:10191600741CE0E0E0930004E0930104E0E0E0934F
:10192600F203E093F303E093F403E093F503E0E0BE
:10193600E093F903219608950E948E1C0E946C1A6A
:101946000E94981C0E9474200E94231B0E949F1CC8
:101956000E94311B0E94A61C10C00E948E1C0E9471
:101966004A1A0E94981C0E9474200E94931A0E9490
:101976009F1C0E94BE1A0E94A61C2A9608952A97AA
:101986000E94982100E010E030E0EFEDF2E00E94C6
:101996004319A12FB0E0EA17FB0710F40C94800D51
:1019A6003230A1F40E94AB1CEB3339F00E94B11C1B
:1019B6000E94AB1CEC930F5F09C00E94B11C0E94F1
:1019C600B81CE0933904F0933A0400E03330A1F4F4
:1019D6000E94AB1CEB3339F00E94B11C0E94AB1C79
:1019E600EC930F5F09C00E94B11C0E94B81CE093E3
:1019F6003B04F0933C0400E03430A1F40E94AB1C9D
:101A0600EB3339F00E94B11C0E94AB1CEC930F5FC4
:101A160009C00E94B11C0E94B81CE0933D04F093DB
:101A26003E0400E03530A1F40E94AB1CEB3339F0E4
:101A36000E94B11C0E94AB1CEC930F5F09C00E9470
:101A4600B11C0E94B81CE0933F04F093400400E0F0
:101A56003A30A1F40E94AB1CEB3339F00E94B11C62
:101A66000E94AB1CEC930F5F09C00E94B11C0E9440
:101A7600B81CE0934104F093420400E03B30A1F42B
:101A86000E94AB1CEB3339F00E94B11C0E94AB1CC8
:101A9600EC930F5F09C00E94B11C0E94B81CE09332
:101AA6004304F093440400E03C3001F50E94AB1C73
:101AB600EB3339F00E94B11C0E94AB1CEC930F5F14
:101AC60015C00E94B11CE0E0EC930E94C01C0E946D
:101AD60031170E94C51C0E94CE1C0E94D71C0E9472
:101AE600861C0E94D2200E94C51C00E00E94AB1CEE
:101AF600EB3309F43F5F1F5F48CFE0914904EF5F86
:101B0600E0934904A0914904A33018F0E0E0E09383
:101B160049040E949F212E9608952C97E4E2E093B3
:101B26005E03E1E30E94DC1CF8940E94EB1C0E9419
:101B3600751778940E942B190E94C01C0E94F21CF3
:101B46000E94F51CE0E0E883A881A63080F40E949C
:101B5600041C0E943C210E94FB1C0E94C01C0E9487
:101B6600F21C0E94F51CE881EF5FE883EDCF0E942E
:101B7600041D0E94C01C0E94F21C0E94F51C0E94BB
:101B86000D1D0E94C01C0E94F21C0E94F51C0E94A2
:101B9600161D0E94C01C0E94F21C0E94F51C0E9489
:101BA6001F1D0E94C01C0E94F21C0E94F51C0E9470
:101BB60006020E942B190E94281D0E942B190E94C2
:101BC600301948F40E943719EA930E946703E881A6
:101BD600EF5FE883F2CFE4E2E0935E03E2E30E9484
:101BE600DC1CF8940E94EB1C0E94751778940E94E6
:101BF6002B190E94C01C0E94F21C0E94F51CE0E0FA
:101C0600E883A881A63070F40E94361C0E94FB1C53
:101C16000E94C01C0E94F21C0E94F51CE881EF5F26
:101C2600E883EFCF0E94041D0E94C01C0E94F21C94
:101C36000E94F51C0E940D1D0E94C01C0E94F21CF1
:101C46000E94F51C0E94161D0E94C01C0E94F21CD8
:101C56000E94F51C0E941F1D0E94C01C0E94F21CBF
:101C66000E94F51C0E9406020E942B190E94281D44
:101C76000E942B190E94301948F40E943719EA93E2
:101C86000E946703E881EF5FE883F2CF2C96089500
:101C9600EF97AD978CE0A0E6B0E0EEECF0E00E94A6
:101CA600A421E0E0E883A881A83040F40E943F1D0B
:101CB600E0E0EC93E881EF5FE883F5CFE091A704DD
:101CC600E03011F00C94BE0FE0E0E883A881A63066
:101CD60010F00C943B0FE881A0911E04AE1710F48F
:101CE6000C942B0F0E943F1D0E94481D0E94041C4D
:101CF6000E943C217F936F93FF93EF930E94F11B09
:101D06000E94221C0E94571DAF91BF918F919F91F7
:101D16000E948C215CF40E945C1D21F40E94611DCE
:101D2600A2E003C00E94611DA1E0A0830E94041CE2
:101D36000E943C217F936F93FF93EF930E94F11BC8
:101D46000E94221C0E946B1DAF91BF918F919F91A3
:101D56000E9491215CF40E945C1D21F40E94611D89
:101D6600A4E003C00E94611DA3E0A0830E94041C9E
:101D76000E943C217F936F93FF93EF930E94F11B88
:101D86000E94221C0E946B1DAF91BF918F919F9163
:101D96000E949121ACF00E94041C0E943C217F937A
:101DA6006F93FF93EF930E94F11B0E94221C0E94E7
:101DB600571DAF91BF918F919F910E948C210CF47A
:101DC6000BC00E945C1D21F40E94611DA5E003C0AA
:101DD6000E94611DAAE2A0830E94701D32960E9495
:101DE600791D3396A0E0A0830E94041C0E947C1DEE
:101DF6000E94851D0E948F1D0E94981D44F40E941A
:101E0600701D33960E94791D3496A0E0A0830E942F
:101E1600A01D0E94B11D0E94701D0E94B41D0E944B
:101E2600041C0E947C1D0E94B71D0E94C11D24F443
:101E36000E94701D0E94CA1D0E94CD1D24F40E949E
:101E4600701D0E94CA1D0E94A01D0E94B11D0CC0DB
:101E56000E943F1D0E94481D0E94701DFA93EA933E
:101E6600E9E3F2E00E94CF1DE881EF5FE8832ECF21
:101E76000E94D31D0E94D81D0E94B11D0E94EC1D18
:101E86000E94F31D0E94FC1D0E94041E0E940D1E4E
:101E96000E94851D0E94D31D0E94121E0E94CD1D08
:101EA60024F40E94D31D0E94121E0E94171E0E9437
:101EB600B11D0E94D31D0E94B41D0E94F31D0E94F5
:101EC600281E0E94171E0E94B11D0E94D31D0E944B
:101ED6002A1E0E942F1E0E948821FCF40E94381E92
:101EE60024F00E94411E0E94481E0E94411EE7E601
:101EF600F1E00E94CF1D0E944E1E0E94581E0E94B5
:101F06006E1E0E94B41D0E944E1E0E94731E24F473
:101F16000E946E1E0E94CA1D1EC00E942F1E0E9495
:101F2600981D24F40E94411E0E94481E0E946E1EA7
:101F36000E94121E0E94851E0E94581E0E946E1E3E
:101F46000E94B41D0E94851E0E94731E24F40E94E6
:101F56006E1E0E94CA1DFE01E05AFF4F01901190AD
:101F660061917081F0010E94871E0E94B11D0E943E
:101F7600411E0E94901EA091A704A13011F00C945E
:101F86000311E0E0E883A881A63010F00C948210DB
:101F96000E943F1D0E94481D0E94041C0E943C2175
:101FA6007F936F93FF93EF930E94F11B0E94221C75
:101FB6000E94571DAF91BF918F919F910E948C21D6
:101FC6005CF40E945C1D21F40E94611DA2E003C026
:101FD6000E94611DA1E0A0830E94041C0E943C2176
:101FE6007F936F93FF93EF930E94F11B0E94221C35
:101FF6000E946B1DAF91BF918F919F910E9491217D
:102006005CF40E945C1D21F40E94611DA4E003C0E3
:102016000E94611DA3E0A0830E94041C0E943C2133
:102026007F936F93FF93EF930E94F11B0E94221CF4
:102036000E946B1DAF91BF918F919F910E9491213C
:10204600ACF00E94041C0E943C217F936F93FF9387
:10205600EF930E94F11B0E94221C0E94571DAF9114
:10206600BF918F919F910E948C210CF40BC00E940E
:102076005C1D21F40E94611DA5E003C00E94611D44
:10208600AAE2A0830E94701D32960E94791D3396A3
:10209600A0E0A0830E94361C0E94931E0E94851D0C
:1020A6000E94CD1D44F40E94701D33960E94791D36
:1020B6003496A0E0A0830E94A01D0E94B11D0E943C
:1020C600701D0E94B41D0E94361C0E94931E0E9421
:1020D600B71D0E94C11D24F40E94701D0E94CA1DD6
:1020E6000E94CD1D24F40E94701D0E94CA1D0E94EC
:1020F600A01D0E94B11DE881EF5FE88344CF0E94D6
:10210600D31D0E94D81D0E94B11D0E94EC1D0E9485
:10211600F31D0E94FC1D0E94041E0E949A1E0E942E
:10212600D31D0E94121E0E94CD1D24F40E94D31DB1
:102136000E94121E0E94171E0E94B11D0E94D31DEE
:102146000E94B41D0E94F31D0E94281E0E94171EA5
:102156000E94B11D0E94D31D0E942A1E0E942F1E9E
:102166000E948821FCF40E94381E24F00E94411E21
:102176000E94481E0E94411EE7E6F1E00E94CF1D24
:102186000E944E1E0E94581E0E946E1E0E94B41D82
:102196000E944E1E0E94731E24F40E946E1E0E9410
:1021A600CA1D1EC00E942F1E0E94981D24F40E9464
:1021B600411E0E94481E0E946E1E0E94121E0E9410
:1021C600851E0E94581E0E946E1E0E94B41D0E940B
:1021D600851E0E94731E24F40E946E1E0E94CA1D54
:1021E600FE01E05AFF4F0190119061917081F0015C
:1021F6000E94871E0E94B11D0E94411E0E94901ED1
:10220600A091A704A23011F00C94CE12E0E0E8836E
:10221600A881A630F8F40E94361CDF01CB01FE012E
:10222600EC59FF4F0190119061917081F0010E946D
:102236008C2164F40E94361CDE01AC59BF4FED932D
:10224600FD936D937C93E881E0931E04E881EF5F34
:10225600E883DECFE0911E04EF5CE887E3E4E987DC
:10226600E5E6EA87ECE6EB87EC87E0E0ED870E949F
:102276009C1E0E94851D0E94A91E0E94B91EE7E2AF
:10228600F1E00E94BE1E0E94CD1D24F4FE0173964D
:102296000E94121E0E94C21EFE0173960E94B41D69
:1022A6000E949C1E0E94B71D0E94A91E0E94C11D6D
:1022B60014F40E94C51E0E94CD1D14F40E94C51E72
:1022C6000E94C21EFE0173960E942A1E0E942F1EA5
:1022D6000E948821CCF40E94C81EE7E6F1E00E9425
:1022E600BE1E0E944E1E0E94CD1E14F40E94DF1ECA
:1022F6000E94E21E0E94F51E0E944E1E0E94731E40
:1023060014F40E94F81E16C00E94C81E0E94481EA1
:102316000E94851E0E94CD1E14F40E94DF1E0E949C
:10232600E21E0E94F51E0E94851E0E94731E14F472
:102336000E94F81EFE01E05AFF4F01901190619134
:102346007081F0010E94FB1E0E94031F0E94C81E9E
:102356000E94901E0E94061F0E94481E0E947D1C1D
:102366000E940B1F10F40E94131F0E947D1C0E94E6
:10237600161F10F40E94131F0E947D1C0E941E1F30
:1023860010F40E94131F0E947D1C0E94261F10F449
:102396000E94131F0E947D1C0E94981D10F40E942B
:1023A600131FE091FA03F091FB036091FC03709117
:1023B600FD030E94FB1EFE01B9960E94B11D0E94FC
:1023C600061FE8E4F2E00E94CF1D0E942E1FEBE4F8
:1023D600F2E00E94BE1E0E94461C0E94882114F054
:1023E6000E94331F0E94461C0E94261F2CF40E9446
:1023F600461C0E94361F0CF402C00E94331F0E9426
:10240600461C0E94981D2CF40E94461C0E943E1FEA
:102416000CF402C00E94331FE0919F04F091A004C7
:102426006091A1047091A2040E94FB1EFE01F49625
:102436000E94B11D0E942E1F0E94461F0E94491F26
:10244600E2E5F2E00E94BE1E0E946B1C0E948821FB
:1024560014F00E944E1F0E946B1C0E94261F2CF433
:102466000E946B1C0E94361F0CF402C00E944E1F75
:102476000E946B1C0E94981D2CF40E946B1C0E94EB
:102486003E1F0CF402C00E944E1FE091A304F0917F
:10249600A4046091A5047091A6040E94FB1EFE018F
:1024A600FF960E94B11D0E94491F0E94461F0E946E
:1024B600EC1D0E94F31D0E94FC1D0E94041E0E943A
:1024C600261F34F40E94D31DFA93EA930E94481EF5
:1024D6000E94D31D0E94D81D0E94B11D0E94EC1DB2
:1024E6000E94F31D0E94FC1D0E94041E0E949A1E5B
:1024F6000E94D31D0E94121E0E94CD1D24F40E942C
:10250600D31D0E94121E0E94171E0E94B11D0E941A
:10251600D31D0E94B41D0E94F31D0E94281E0E9416
:10252600171E0E94B11D0E94D31D0E942A1E0E94E2
:10253600411EE6E5F2E00E94BE1E0E94511FA03138
:10254600E7E2BE0720F40E946E1E0E94121E0E9441
:10255600511FA83EE3E0BE0720F40E946E1E0E94B3
:10256600121E0E94511FA436E0E0BE0720F40E940E
:102576006E1E0E94121E0E94511F1A9720F40E947E
:102586006E1E0E94121EE091F603F091F7030E9460
:10259600561F0E94B11DA091A704A33011F00C9400
:1025A6008D140E945F1FEBE5F2E00E94BE1E0E94A2
:1025B600641F0E946B1F0E94CD1D24F4FE013896F5
:1025C6000E94121EFE0138960E94B11DFE01389629
:1025D6000E94B41D0E94641F0E94771F0E94CD1D99
:1025E60024F4FE0138960E94CA1DFE0138960E9408
:1025F600B11DFE0138960E942A1E0E94B91EEFE503
:10260600F2E00E94BE1E0E94831F0E946B1F0E9462
:10261600CD1D24F4FE0173960E94121E0E94C21E56
:10262600FE0173960E94B41D0E94831F0E94771FAD
:102636000E94CD1D14F40E94C51E0E94C21EFE01FA
:1026460073960E942A1E0E94C81EE3E6F2E00E94CC
:10265600BE1E0E948A1F0E946B1F0E94CD1D14F48D
:102666000E94DF1E0E94031F0E94F51E0E948A1F01
:102676000E94771F0E94CD1D14F40E94F81E0E942E
:10268600031FFE017E960E942A1E0E94061F0E94BC
:10269600481E0E94CE1C0E940B1F10F40E94131F9E
:1026A6000E94CE1C0E94161F10F40E94131F0E9447
:1026B600CE1C0E941E1F10F40E94131F0E94CE1CE7
:1026C6000E94261F10F40E94131F0E94CE1C0E9417
:1026D600981D10F40E94131FE0914504F0914604E2
:1026E60060914704709148040E94FB1EFE01B99652
:1026F6000E94B11D0E94061FE8E4F2E00E94CF1D71
:102706000E942E1FEBE4F2E00E94BE1E0E94911F63
:10271600109714F00E94331F0E94911FA436E0E028
:10272600BE073CF40E94911FECE9FFEFEA17FB0796
:102736000CF002C00E94331F0E94911F1A973CF4AE
:102746000E94911FE6EFFFEFEA17FB070CF002C0AD
:102756000E94331FE0914104F09142040E948A20B6
:102766000E94FB1EFE01F4960E94B11D0E942E1FC0
:102776000E94461F0E94491FE2E5F2E00E94BE1E2B
:102786000E94961F109714F00E944E1F0E94961FDB
:10279600A436E0E0BE073CF40E94961FECE9FFEF8A
:1027A600EA17FB070CF002C00E944E1F0E94961FFC
:1027B6001A973CF40E94961FE6EFFFEFEA17FB0715
:1027C6000CF002C00E944E1FE0914304F0914404B5
:1027D6000E948A200E94FB1EFE01FF960E94B11DE8
:1027E6000E94491F0E94461F0E94EC1D0E94F31D75
:1027F6000E94FC1D0E94041E0E94261F34F40E94A3
:10280600D31DFA93EA930E94481E0E94D31D0E948C
:10281600D81D0E94B11D0E94EC1D0E94F31D0E944E
:10282600FC1D0E94041E0E949A1E0E94D31D0E9437
:10283600121E0E94CD1D24F40E94D31D0E94121E5A
:102846000E94171E0E94B11D0E94D31D0E94B41D36
:102856000E94F31D0E94281E0E94171E0E94B11D91
:102866000E94D31D0E942A1EE0914904E03091F097
:10287600E13039F40E94D31DFA93EA93EAE6F2E0D6
:1028860011C0E23039F40E94D31DFA93EA93EDE6C3
:10289600F2E008C0FE013896EE5BFF4FFA93EA932A
:1028A600E7E6F2E0FA93EA930E9424200E94411E92
:1028B600E6E5F2E00E94BE1E0E949B1FA031E7E201
:1028C600BE0720F40E946E1E0E94121E0E949B1FCD
:1028D600A83EE3E0BE0720F40E946E1E0E94121E70
:1028E6000E949B1FA436E0E0BE0720F40E946E1EE5
:1028F6000E94121E0E949B1F1A9720F40E946E1EB1
:102906000E94121EE0913904F0913A040E94561F6B
:102916000E94B11DA091A704A43001F50E945F1F7B
:10292600E0E7F2E00E94BE1E0E94C81EEAE7F2E05F
:102936000E94BE1E0E94D31D0E94D81D0E94B11D7A
:102946000E94AB190E94B01921F0A091E203A037B2
:1029560009F004C00E94B6190E948609E0E00E94B0
:102966009A1B0E945F1F0E94AE18FE0138960E94B5
:102976004319E883A881AA3030F40E94DA1AE88164
:10298600EF5FE883F7CFEAE00E949A1B0E94B91E28
:102996000E94AE18FE0173960E944319E883A8812F
:1029A600AA3030F40E94DA1AE881EF5FE883F7CFA5
:1029B6000E94F3190E94C81E0E94AE18FE017E9660
:1029C6000E944319E883A881AA3030F40E94DA1ADB
:1029D600E881EF5FE883F7CFEAE00E949F1B0E9441
:1029E600061F0E94AE18FE01B9960E944319E8839D
:1029F600A881AA3030F40E94DA1AE881EF5FE883F2
:102A0600F7CFE0E00E94A01F0E942E1F0E94AE1882
:102A1600FE01F4960E944319E883A881AA3030F497
:102A26000E94DA1AE881EF5FE883F7CFEAE00E94B6
:102A3600A01F0E94491F0E94AE18FE01FF960E9429
:102A46004319E883A881AA3030F40E94DA1AE88193
:102A5600EF5FE883F7CFE0E00E94B21B0E94D31D30
:102A6600FA93EA930E94AE180E94D31D0E9443195E
:102A7600E883A881AA3030F40E94DA1AE881EF5F71
:102A8600E883F7CFEAE00E94B21B0E94411E0E9433
:102A9600AE180E946E1E0E944319E883A881AA30D0
:102AA60030F40E94DA1AE881EF5FE883F7CFEF96F9
:102AB600AD96089510E0E0E0E093E603E093E703C7
:102AC600E093E803E093E903E0E0E093EA03E093B0
:102AD600EB03E093EC03E093ED03E0E8EBBBE0EC03
:102AE600EABBE4EAE8BBE7EAE7BBE0E0E5BBEFEF19
:102AF600E4BBE0EFE2BBE0E0E1BBE3E0E3BFE0E044
:102B0600E2BFECBFEFBDEAE0EEBDE0E0EDBDECBD3F
:102B1600E7BDE6BDE3ECEBBDEFE4EABDE0E0E9BD11
:102B2600E8BDE2BDE5BDE4BDE3BDEBB7E06CEBBFE0
:102B3600EBE0E5BFE0E0E4BFE0ECEABFE1E1E9BFDE
:102B4600E0E0EBB9E8E5EAB9E6E8E0BDE0E0E0BDE3
:102B5600E9E1E9B9E0E8E8B9E0E0E0BFE0ECE7B9CF
:102B6600E3E8E6B90E940A19E4E00E94A51FE8E03E
:102B76000E94A51FE0E00E949A1BE4E8F2E00E9492
:102B8600EF190E948518A0E0B0E00E945D210E9426
:102B9600281BA2E0B0E00E945D210E943F1AA4E03B
:102BA600B0E00E945D210E94981AA6E0B0E00E9463
:102BB6005D21E0932D04F0932E04A8E0B0E00E947E
:102BC6005D210E945B1BAAE0B0E00E945D210E948D
:102BD600651BACE0B0E00E945D21E0933304F09306
:102BE6003404AEE0B0E00E945D21E0933504F0933A
:102BF6003604A0E1B0E00E945D210E943D1BA3E1E6
:102C0600B0E00E945D210E94C31B0E94C81BE4E63F
:102C1600F0E00E94BA20E09305040E94C81BE4E697
:102C2600F0E00E94FC20E0930404A5E1B0E00E94DD
:102C36006121E093DF03A2E1B0E00E946121E0930D
:102C4600E103E093A704E89423F8A091A704A53034
:102C560018F0E0E0E093A704C59AC79ADF9A0E94AD
:102C6600CF1F0E94FA04C29AE1E0F0E00E94921996
:102C76000E9489030E94F2017894E3E00E949A1B65
:102C8600EFE9F2E00E94EF19E4E00E949F1BEEEAF2
:102C9600F2E00E94EF19E4E00E94A01FE9EBF2E0E7
:102CA6000E94EF19E4E00E94B21BE2ECF2E00E94FF
:102CB600EF190E94F9190E94AB19A091E203A03EF8
:102CC60011F40E9453050E94FC190E94AB190E9440
:102CD600B019B9F00E94B619E091E203E03D39F46B
:102CE6000E94BB1918F0E0E0E093A70408C0E03B9F
:102CF60031F40E94C41919F4E4E0E093A7040E9499
:102D06004B0EE0E021FCE1E0E13010F40C94D31628
:102D16000E943205E1E0EA930E945404E093210404
:102D2600F0932204A0912104B0912204A433E2E09E
:102D3600BE0724F0A53BE1E0BE075CF00E940B1A3B
:102D4600E0931F04F0932004FA93EA930E94B00CD8
:102D560008C0E0912104F0912204FA93EA930E94BC
:102D66009F0CE0932304F09324046093250470934E
:102D760026040E94E60A0E944B0EE0E023FCE1E0F6
:102D8600E13060F00E94900DE091F603F091F703B8
:102D96003196E093F603F093F7033197E89421F820
:102DA600E0E020FCE1E0E130A8F0E89420F810E053
:102DB600EFEDF2E00E944319A12FB0E0AE17BF0776
:102DC60038F40E94AB1CEA930E9467031F5FF0CFA2
:102DD6000E94C20CA091E003A23038F00E94CF1FDF
:102DE6000E94FA04E0E0E093E0036FCFFFCF5F9B21
:102DF600FECFECB10895B981A881EC91EA930E94C7
:102E0600FD1FEE2311F01196F8CFE894EC91ED3208
:102E160011F4689402C0EB3209F4119666277727FD
:102E2600EC91EA930E94F51FEE2381F0E62FF72F2F
:102E3600660F771F660F771F6E0F7F1F660F771F50
:102E4600ED91FF27E0536E0F7F1FEACFE62FF72F96
:102E56001EF4E095F095319622960895B981A881E1
:102E6600EC91EA930E94FD1FEE2311F01196F8CF24
:102E7600E894EC91ED3211F4689402C0EB3209F457
:102E860011960024112488279927EC91EA930E9431
:102E9600F51FEE2399F0E02DF12D682F792F1DD027
:102EA6001CD00E0E1F1E861F971F17D0ED91FF27F1
:102EB600E0530E0E1F1E8F1F9F1FE7CFE02DF12D33
:102EC600682F792F46F4E095F095609570958827E0
:102ED6003196681F781F22960895000C111C881FD2
:102EE600991F0895A991B991E991F99130962AF41B
:102EF600E095F09531966DE26D93E89480E197E266
:102F06000DD088EE93E00AD084E6992707D08AE0B0
:102F160005D06E2F10D066276C9308956627E817A4
:102F2600F90720F06395E81BF90BC9F7662311F43E
:102F360016F008956894605D6D93089524971A932A
:102F46000A93E0E0FAEC6AE97BE3EA83FB836C83AD
:102F56007D8300E00E94D41F0E94882174F4E885D6
:102F6600F9856A857B850E947D20E887F9876A87CF
:102F76007B870E94D91FEDE2EC930E94E01F0E941E
:102F8600D2201E2F103071F4003061F4AA81BB816B
:102F96008C819D81A130E0E0BE07E0E08E07E0E095
:102FA6009E0731F40E94D91FE12FE05DEC9301E00A
:102FB6000E94E01F0E94FF20E887F9876A877B87C7
:102FC600AA81BB818C819D810E940D1E0E94D22008
:102FD600EA83FB836C837D830E94842171F6AE8134
:102FE600BF81E0E0EC93198108812C960895FFE0FB
:102FF600FA95F1F70895AFE0A4BBA99AA898A5B3EE
:10300600B091A8050E94FA17AB2BA5BB0E94FA1730
:10301600E3B3A37FA5BB0E94FA17AB2BA5BB0E9407
:10302600FA17A37FA5BB0E94FA17E7FDEBCF089519
:10303600A07FAB2BA5BBAE2BA5BB0E94FA17A37F27
:10304600A5BB0E94FA170895A998AFEFA4BBE0911B
:10305600A805B5B3BF70A8810E941B18A881A295C8
:103066000E941B18A99A219608950E94FE17E981CD
:103076000E94E51FA89AE881EA930E9427182296E3
:103086000895B5B3E091A805BE2BB5BB0E94FA170B
:10309600E3B3B37FB5BB0E94FA17E07F08950E94A1
:1030A600FA170E944418AE2F0E944418A998E29578
:1030B600EA2B08951A93E4E0E093A805A981A230CB
:1030C60018F0E8E0E093A805EA81E0581E2FE981B0
:1030D600E17009F010640E94FE171A930E942718E7
:1030E600BA80A9801881239608950E94FE17E2E00F
:1030F6000E94E51FECE00E94E51FE1E0EA930E94D2
:1031060027180895E8E0E093A8050E947818E4E0FF
:10311600E093A8050E947818E0E0AE2EBE2E089532
:10312600EF93FF93A8816894AA3029F0E894B394AA
:10313600E8E2EB1538F4A394E0E0EA93AA920E9441
:103146005D182EF058DFA89AA881AA937DDFFF911B
:10315600EF91219608951A93A981BA81ED91A983D9
:10316600BA831E2FE03021F01A930E949318F4CFF1
:10317600188110C01A93E981FA813196E983FA839E
:103186003197E4911E2FE03021F01A930E94931894
:10319600F2CF188123960895AA27BB271197F1F736
:1031A6000895A998AFEFA4BBE091A805B5B3BF7089
:1031B600A8810E941B18A99A219608950E94EA1FC9
:1031C6000E94EA1F0E94EA1F0E94CF18E0E2EA93DB
:1031D6000E94D4180E94CF18E8E20E94F01FE4E093
:1031E6000E94F01FE5E80E94F01FA4B3AF70A4BBD5
:1031F600A99A0E945218E53011F0E0E008950E9465
:10320600FE17E6E0EA930E942718E1E00895AA98DF
:10321600AB98A898E4E0E093A8050E94E118E03096
:1032260011F4E0E00895E8E0E093A8050E94E118B3
:10323600E03011F4E0E008950E948518E1E0089579
:10324600EEECEA930C94CA01E9E8EA930C94CA01FD
:10325600EEE5F3E0FA93EA9308950E944920A881E7
:10326600B0E0AE17BF070895E881F0E0E25AFC4FE0
:10327600E0810895FE013396FA93EA930C941520A3
:10328600FA93EA930C944920F0E0E05AFD4FE0816E
:1032960008950A921A92FA926A937A938A939A9363
:1032A600AA93BA93EA93FA93EFB7EA930895E09153
:1032B600DD03F0E0E05AFD4F0895FA93EA930C948B
:1032C6003320E991EFBFF991E991B991A9919991CB
:1032D600899179916991F990199009900895E091F1
:1032E600DF03ACE7B0E0F0E0EE0FFF1FEA0FFB1FD5
:1032F6000895E0ECEA930C94CA01A091F203B09110
:10330600F3038091F4039091F5030895E093F2039B
:10331600F093F3036093F4037093F5030895FA931F
:10332600EA930C945E20C598E0E1EA930E947F043C
:10333600E8E1EA930C947F04C598E8E0EA930C94DC
:103346007F04EA930E947F04E4E0EA930C947F04EE
:103356000E946D04E093E2030895E091E303A091D7
:10336600E203EA170895E091E203E093E303089588
:10337600E091A704EF5FE093A704A091A704A5300E
:103386000895E091A704E150E093A704EF5F089544
:10339600E2E3F0E0C4CFE091E003EF5FE093E00307
:1033A600E1500895A2E1B4E0F0E0EE0FFF1F0895AA
:1033B600E12FA6E0B4E0F0E0EE0FFF1F0895AE0F98
:1033C600BF1F0E943821D00108950E948518E0E0B1
:1033D600EA93EA930C945D18FA93EA930C94BD1859
:1033E600E0E0EA93E1E0EA930C945D18E8EEF3E09E
:1033F60096CFE0EFE093E203B6CFE0E0E0932D0452
:10340600E0932E04E0E0E0932904E0932A04089573
:10341600E0E0EA930C9454049F01E1E0EA930E94F1
:103426005404AF01F901A0912D04B0912E04EA0FC6
:10343600FB1FE0932D04F0932E04FA01A0912904BA
:10344600B0912A04EA0FFB1FE0932904F0932A04A3
:103456000895A0912D04B0912E040895EAE0F0E0BD
:103466000E94CD200895E0932D04F0932E04A091A0
:103476002904B0912A04F2CFE0932904F0932A0498
:103486000895E5E0EA93E1E0EA930C945D18E09193
:103496002D04F0912E040895FA93EA93FE013E96C8
:1034A600FA93EA930E947517FE013C96FA93EA9303
:1034B6000895FA93EA930E942420FE013C96FA931B
:1034C600EA930C94AE18E5E0EA93E2E0EA930C94F2
:1034D6005D18E0912904F0912A040895A6E0B0E071
:1034E6000E945D21B6DFEA17FB070895A2E0B0E06F
:1034F6000E945D21A0912904B0912A04EA17FB07D6
:103506000895C5DFA6E0B0E00E946D210895E1DFD1
:10351600A2E0B0E00E946D210895E7E3F1E05CCF00
:10352600E0912B04F0912C040895E0932B04F09382
:103536002C04089566277727E8A3F9A36AA37BA33B
:103546000895A8A1B9A18AA19BA10E948A200895E5
:103556000E947420A8A3B9A38AA39BA308950E94DE
:10356600B520E8A3F9A36AA37BA30895A8A1B9A1EE
:103576008AA19BA10895E0EAF0E060E070E00E9475
:10358600F7200895E8A3F9A36AA37BA37ACFEDE514
:10359600F1E08FCFEBDF0E9488210895E7E6F1E0A6
:1035A6001BCFE4DFEFEFFFEF6FEF7FEFD8CFE8E25F
:1035B600F1E012CFDBDFE4E6F0E060E070E00895D2
:1035C6000E94F720AF01E6E0EA93E2E0EA930E9468
:1035D6005D184930E0E05E070895E7E0EA93E2E02F
:1035E600EA930C945D185A934A93FE013896FA931F
:1035F600EA930E947517FE013C96FA93EA93FE0140
:1036060038960895FE013C96FA93EA930895E9E602
:10361600F1E0FA93EA930E942420CCCF0E94032182
:10362600AF014A30E0E05E070895EBE6F1E0FA9379
:10363600EA930C942420FA93EA930E941520E2CF91
:10364600E0912704F09128040895E0932704F0936D
:1036560028040895EA930E9454046CCFE0E1F0E058
:1036660060E070E00E94F7200895E0913704F09141
:1036760038040895E0933704F09338040895E0E0A1
:10368600F2E060E070E00E94F72008956FDFEAE064
:10369600F0E060E070E00895E6E0EA93E2E0EA93A5
:1036A6000C945D18E9E6F1E0FA93EA930C94242071
:1036B600E0932F04F09330040895E0913104F091E3
:1036C60032040895E0933104F09332040895E1E062
:1036D600EA93EA930C945D18E0912F04F09130047C
:1036E60008950E94AE18E9EBF1E076CEE1E0EA93A8
:1036F600E2E0EA930C945D1839DFE2E2F1E060E083
:1037060070E02DCFE0913304F09134040895E8A1E0
:10371600F9A1FA93EA93FE013896FA93EA930E9486
:10372600751770CFE0913504F09136040895EA9349
:10373600E0E0EA930C945D18EA93E1E0EA930C94D6
:103746005D18F0E0FA93EA93FE013296FA93EA9353
:103756000E947517FE01FA93EA930C94AE18EA9349
:10376600E3E0EA930C945D1823F8E0E0E093F603B7
:10377600E093F7030895E0930404A09104040895E8
:10378600E0930204F09303040895A0910204B0911B
:1037960003040895E0910204F09103040895E8817A
:1037A600AAE4B4E0F0E00E948520EA0FFB1F08952A
:1037B6000F01E881A6E0B4E0F0E0EE0FFF1FFFCDB9
:1037C6000E944221E881A6E6B4E0F0E00E9485204E
:1037D6000895662777270E9442210895E881A2E886
:1037E600B4E0F0E00E9485200895E881E150A6E665
:1037F600B4E0F0E00E948520AE0FBF1F0E943C217E
:103806000895E881A6E6B4E0F0E00E948520AE0FB8
:10381600BF1F0895E881A6E6B4E0F0E00E94852087
:10382600EA0FFB1F0895E881E150A2E8B4E0F0E05A
:103836000E948520AE0FBF1F0E943C210895AE0F47
:10384600BF1F0E943C210895A7E2BAE680E090E0FF
:103856000E94B520DF01CB01E0E0F0E860E070E017
:103866000E94F7200895E881AAE4B4E0F0E00E94FF
:103876008520E5CFE0939F04F093A0046093A10414
:103886007093A2040895A0919F04B091A004809122
:10389600A1049091A2040895AF3FE3E0BE07E0E0E3
:1038A6008E07E0E09E0708950E948A200E947420F9
:1038B600E2E2F1E060E070E00E94B5200895E09356
:1038C600A304F093A4046093A5047093A60408953A
:1038D600A091A304B091A4048091A5049091A6049C
:1038E6000895E093FA03F093FB036093FC0370934F
:1038F600FD030895A091FA03B091FB038091FC03A8
:103906009091FD0308950E948F20DF01CB0142DFD5
:103916006627772708952897E885F9850E948A20E3
:10392600E883F9836A837B830895A881B9818A81B4
:103936009B810E948A2008950E948A200E94B520B9
:10394600DF01CB010895EC83FD836E837F830895A9
:10395600E12FF0E0E152FD4FE0810895E02FF0E025
:10396600DE011496AE0FBF1F0895E0E0EC93FE0152
:103976003496FA93EA930C94FE16FE013496FA9363
:10398600EA930895E0934504F09346046093470450
:10399600709348040895A0914504B091460480911F
:1039A6004704909148040895E4E6F0E060E070E092
:1039B6000895E0935F03EBE3E0936003E1E3E093B4
:1039C6006103EBE3E0936203E0E0E09363030895B1
:1039D600E091F603F091F703FA93EA93CECF0E94B3
:1039E600152036CCE7E3F2E0FA93EA930C94242010
:1039F6000E944B21FE013696FA93EA930E94A11784
:103A060027CCE0912304F091240460912504709161
:103A16002604EECFE0919F04F091A0046091A104EA
:103A26007091A204E5CFE091A304F091A404609103
:103A3600A5047091A604DCCFE091FA03F091FB0394
:103A46006091FC037091FD03D3CF0E944920E98366
:103A5600F0E0E25AFC4FADE0A083E981F0E0E15AE4
:103A6600FC4FAAE0A083E981F0E0E05AFC4FA0E019
:103A7600A083E0E0E8830895E881ABE0EA9FF001E7
:103A8600DE011896AE0FBF1F0895E881EF5CEC9338
:103A9600E881ABE0EA9FF001DE011896EA0FFB1F12
:103AA6003196A0E0A0830895EB5FFF4F6F4F7F4FE5
:103AB6000895E881A0919E04EA170895E881ABE095
:103AC600EA9FF001DE011896EA0FFB1F3196089572
:103AD600E550F040604070400895E881ABE0EA9F11
:103AE600F001DE011896EA0FFB1F0895A0E2A083FD
:103AF600F4CF0E943C21DF01CB01E8EEF3E060E069
:103B060070E008950E94F720DE01A859BF4FED939B
:103B1600FD936D937C930895DE01A859BF4F0D90D8
:103B26001D908D919C91D0010895AA30E0E0BE07CA
:103B3600E0E08E07E0E09E070895FE01E859FF4F9A
:103B46000190119061917081F0010E944B21FE015C
:103B56003596FA93EA930E94A117BFCFFA93EA9398
:103B660089CBFA93EA939ECD0E940321DE01A859E0
:103B7600BF4FED93FD936D937C930895CDDFA436EF
:103B8600E0E0BE07E0E08E07E0E09E070895FA93C6
:103B9600EA934BCDC1DFC9CFFA93EA930C94242064
:103BA600FE013896EE5BFF4F0895FA93EA93E2E43E
:103BB600F2E0FA93EA930E943E20E091A704F0E037
:103BC600FA93EA93FE013396FA93EA930E947517E5
:103BD600E7CFE4E0EA930E945404A2E6B4E0F9CD0C
:103BE600A0916204B091630480916404909165048D
:103BF60008953BDD662777270E94B520DF01CB01BC
:103C06003ECDE0936204F093630460936404709382
:103C16006504E6CFEAE0F0E060E070E00895FA932C
:103C2600EA93E8E2F1E0B8CFFE01E859FF4F0190D0
:103C3600119061917081F0010E944B21FE01359631
:103C4600FA93EA930E94A117ABCFE4DF8DCFFA93E4
:103C5600EA93E4E4F2E0A0CFA0912304B091240417
:103C660080912504909126040895F6DFA73FEFEF93
:103C7600BE07EFEF8E07EFEF9E070895FE01389619
:103C8600E35BFF4FFA93EA930895E8E2F1E0FA93D3
:103C9600EA930C943E20E0DFEFEFFFEF6FEF7FEF4C
:103CA6000E94B520DF01CB017FCE0E94F720DE0106
:103CB600A05ABF4FED93FD936D937C930E944B21C9
:103CC600FE013596FA93EA930E94A117FE013896F3
:103CD600E35BFF4F43CFFE013896E35BFF4F08954A
:103CE6000E940321DE01A05ABF4FED93FD936D9311
:103CF6007C93DE01A05ABF4F0D901D908D919C9133
:103D0600D00113CFA9DF50CE0E944B21FE0135967C
:103D1600FA93EA930E94A117DECFE6E4F2E03CCFE5
:103D2600DF01CB01E8EEF3E060E070E0089572DFBA
:103D3600E9CEDE01AC59BF4F0D901D908D919C913F
:103D4600D001E8EEF3E060E070E00895FE01E85986
:103D5600FF4F0190119061917081F0010E944B21FB
:103D6600FE013596FA93EA930C94A117FE01739619
:103D7600FA93EA930895FA93EA930C943E20FE018F
:103D86007396ECCEFE01739602CFFE017E96FA93F1
:103D9600EA9308950E94F720DE01A05ABF4FED93E3
:103DA600FD936D937C93DE01A05ABF4F0D901D903D
:103DB6008D919C91D001B9CEFE017E9630CFFE0149
:103DC600E05AFF4F0190119061917081F0010E94BD
:103DD6004B21FE013596FA93EA930E94A117FE0144
:103DE6007E96BCCEFE017E96BCCEFE017E96CFCEE2
:103DF6000E944B21FE013596FA93EA930C94A11783
:103E0600FE017E96ABCEFE01B996FA93EA9308952B
:103E1600A03AE6E8BE07E1E08E07E0E09E070895D7
:103E2600FE01B996FCCEA031E7E2BE07E0E08E07C0
:103E3600E0E09E070895A83EE3E0BE07E0E08E07B7
:103E4600E0E09E070895A436E0E0BE07E0E08E07B6
:103E5600E0E09E070895FE01F496FA93EA9308952A
:103E6600FE01F496DCCEAD39EFEFBE07EFEF8E071D
:103E7600EFEF9E070895A73FEFEFBE07EFEF8E0720
:103E8600EFEF9E070895EFE4F2E086CEFE01FF967F
:103E9600FA93EA930895FE01FF96C1CEA091F60328
:103EA600B091F7030895FA93EA93FE013396FA93D5
:103EB600EA930E9475170FCFFE013896FA93EA939C
:103EC6000895A0913B04B0913C04E4E6F0E0089527
:103ED6000E94BA2066277727DE01A859BF4FED93C7
:103EE600FD936D937C9332CF0E94FC206627772743
:103EF600DE01A859BF4FED93FD936D937C9326CFBA
:103F0600A0913D04B0913E04E4E6F0E00895A0914E
:103F16003F04B0914004E4E6F0E00895A091410426
:103F2600B09142040895A0914304B09144040895C9
:103F3600A0913904B0913A040895EA93E2E0EA9335
:103F46000C945D18E093A805E4E5F0E0FA93EA9393
:103F5600E1E0EA930E949E01ECE5F0E0FA93EA9331
:103F6600E2E0EA930E949E01E4E6F0E0FA93EA9327
:103F7600E3E0EA930E949E01ECE6F0E0FA93EA930E
:103F8600E4E0EA930E949E01E4E7F0E0FA93EA9304
:103F9600E5E0EA930C949E010E94EB04E1E0F0E078
:103FA600BEC9A885B9858A859B850895AE81BF81DE
:103FB6001196AE83BF8311970895EA81FB816C81C8
:103FC6007D81EFCFEA930E9427180C94FE170E947A
:103FD600CF18E0E3EA930C94D418EA930E942718CA
:103FE6000C94CF18E1E0F991F03310F0FA3308F0B1
:103FF600EE270895E1E0F991F03229F0F93010F05A
:10400600FE3008F0EE270895E1E0F991F05340F014
:10401600FA3038F0FF75F750FA3010F0F03108F04A
:10402600EE270895E991F991A991B991CD016D9184
:104036006623E9F7119761916D936623E1F7FC0119
:104046000895E991F991A991B991CD016D916623F0
:10405600E9F7119705900D920020E1F7FC0108950C
:10406600E991F991A991B991CD0161916D93662379
:10407600E1F7FC010895E991F991A991B991CD0172
:1040860005900D920020E1F7FC010895A991B991E0
:10409600EE27FF276D91662311F03196FBCF089529
:1040A600AA27BB27E991F9910590002011F01196F6
:1040B600FBCFFD010895E991F991309639F080EA38
:1040C6009FE00197F1F7A8953197C9F70895EA0F90
:1040D600FB1F681F791F0895EA1BFB0B680B790B02
:1040E6000895AE1BBF0B860B970B0895F195E195CE
:1040F600F0400895F09560957095E195FF4F6F4FEC
:104106007F4F0895EE0FFF1FEE0FFF1F08956F2FCD
:10411600660F660B762F08957A9F702D6B9F700D34
:10412600F89F700DE99F700D6A9F602D710DFB9FC2
:10413600600D711DE89F600D711D8827FA9FF02D97
:10414600610D781FEB9FF00D611D781FEA9FE02D32
:10415600F10D681F781F08956E2F6A9FF0016B9FFF
:10416600F00D08956FD0D8DF0EF4C4DF0895002453
:10417600112490E1AA0FBB1F001C111C0E1A1F0A66
:1041860018F40E0E1F1E01C0A1609A9599F7FD0145
:10419600D001089549D0EBDF0EF4A8DF08953F93D0
:1041A6004F935F93002411244427552730E2AA0F2A
:1041B600BB1F881F991F001C111C441F551F0E1A78
:1041C6001F0A460B570B28F40E0E1F1E461F571FBD
:1041D60001C0A1603A9559F7FD01BC01D001CA01A1
:1041E6005F914F913F9108952DD0D9DF0EF482DF74
:1041F6000895BDDFFD010895D2DFFD01BC010895DC
:10420600E89497FF09C0A095B09580959095AF5F0B
:10421600BF4F8F4F9F4F689477FD6CDFC0DFFD0166
:10422600BC010EF467DF0895E894F7FF02C05EDF75
:104236006894B7FF06C0A095B095119600F8039450
:1042460000FA0895E89477FF02C054DF689497FF58
:104256000BC00024A095B095809590951196801D71
:10426600901D00F8039400FA0895ED91FC911197C2
:104276000895ED91FD916D917C9113970895ED93BD
:10428600FD936D937C9308950590F491E02D089528
:104296007A936A93FA93EA930895182E862F612DDE
:1042A600192E972F712D1B2EBF2FF12D1A2EAE2FE3
:1042B600E12D0895119602D0FE2F1197E199FECFB8
:1042C600FF93FFB7F894AEBBBFBBE09AEDB3FFBF59
:1042D600FF91089507D01196EF93EF2F03D0EF913A
:1042E60011970895E199FECF9FB7F894AEBBBFBB77
:1042F600E09A8DB3E81719F0EDBBE29AE19A9FBFF9
:10430600089530976040704008951097804090401F
:104316000895EA17FB07680779070895AE17BF07E0
:104326008607970708955A934A933A932A931A93BE
:104336000A9308955D814C813B812A811981088108
:104346000895AC0FBD1F05900D928A95E1F708956B
:00000001FF
